:080000001F308A00602F000090
:10002000FF00030E8301A1000A08A0008A01040852
:10003000A2007708A3007808A4007908A5007A0830
:10004000A600831383128C308400801E29288C1A0A
:100050003A28220884002308F7002408F80025081D
:10006000F9002608FA0020088A00210E8300FF0EFE
:100070007F0E09008A110A123D288C1E3D2818089F
:10008000A7001A08F800A71C4728181218167808A5
:100090008316B90083120C1E4B2899008C128A110A
:1000A0000A1229280D050D0523104226EF30E432EF
:1000B0007210381C3710A82129103218B119A02548
:1000C000C125CC060A002310D232F332723B6532CE
:1000D0003A102526F5060A0023104626C129C82F06
:1000E0004529C129C52FD324DA223A102526F50641
:1000F0000A0023104626C129C82F5729492AC52F8F
:10010000D324DA223A102526F5060A002310C23736
:100110006F3A2026EF30E4327210D432733A201F47
:100120003E1F0D05231000015F08E1005E08E0009E
:100130006108FA006008840083137A188317800826
:100140000319A628E00A0319E10A98285E0860024C
:10015000F7006108FA005F08031C5F0FFA027708D6
:10016000F8000800831603178C170C140000000019
:1001700083120C087F390319F8280313DE000317D4
:100180000D080313DF0003170F080313E0005E08D8
:100190000C1EC82899005F0803178D000313600820
:1001A00003178F0083168C170C14000000008312B5
:1001B0000C0D0E0D7F390319F8280313DE00031709
:1001C0000D080313DF0003170F080313E0005E0898
:1001D0000C1EE82899005F0803178D0003136008C0
:1001E00003178F008D0A03198F0A0313B228031710
:1001F00003130800831603178C170C14000000006B
:1002000003182A2983120C087F390313AD00031742
:100210000D080313AE0003170F080313AF002D08DA
:100220000C1E102999002E0803178D0003132F08A8
:1002300003178F0083168C170C1400000000831224
:100240000313AC0B24292729831603172A294A29CB
:100250008316031783120C0D0E0D7F390313AD00A7
:1002600003170D080313AE0003170F080313AF00A5
:100270002D080C1E392999002E0803178D00031331
:100280002F0803178F008D0A03198F0A0310031319
:10029000AC0BFA280800B4010408B3003410831B27
:1002A00034142D0EF038AF00AF07E23EB000323EFE
:1002B000B2002D080F39B007B007B207E93EB10010
:1002C000B107B1072C0E0F39B107B207B10DB20D4E
:1002D000B209B20D2C080F39B207AF0D0730AE00CE
:1002E0000A30B207B103031C7129B107B003031C24
:1002F0007529B007AF03031C7929AF07AE03031CB0
:100300007D292E308400831307303305331384078F
:1003100032300402031933170008F700031D98292F
:10032000331B9829331AA029B319982920309B2907
:10033000B31533123030F70777080C1E9D2999004A
:10034000840A331F882908003008F8012F02031897
:10035000AC292F08F700B829F7010830B100AF0D1C
:10036000F70D300877020318F700F80DB10BAF292D
:100370000800AB012708AB002430AC004930AD00C9
:100380006430AE003A30AF002030B0006230B100CF
:100390006C30B2006F30B3006130B4006430B5002F
:1003A0006530B6007230B7002E30B8006330B90047
:1003B0002030BA003230BB003830BC003430BD00D1
:1003C0003830BE002030BF003230C0003030C100B5
:1003D0003130C2003330C3002D30C4003030C5008E
:1003E0003330C6002D30C7003230C8003130C9006C
:1003F0002030CA003030CB003830CC003A30CD004D
:100400003130CE003630CF003A30D0003430D10019
:100410003930D2005A30D3002030D4006B30D500B0
:100420006130D6006B30D7006C30D8002030D90056
:100430002430DA00DB01DF012C30DE0094200130B3
:1004400078022C3E840083130008243C031D322ACA
:10045000DF012C30DE009420013078022C3E840035
:1004600083138001523003178D0000308F00031377
:10047000B22023300C1E3A2A9900303084008313B6
:1004800080080319562ADF010408DE005F10831B71
:100490005F1400080C1E4A2A99005E08840083132A
:1004A0005F188317840A0319850A402A0D300C1E31
:1004B000572A99000A300C1E5B2A990063300317F3
:1004C0008D0000308F0003100C300313AC00FA20B5
:1004D000103084000330AD001030AC004B210D30E3
:1004E0000C1E702A99000A300C1E742A99006C3078
:1004F00003178D0000308F00031014300313AC007D
:10050000FA2010308400AD012030AC004B210D30BA
:100510000C1E882A99000A300C1E8C2A990079300A
:1005200003178D0000308F00031014300313AC004C
:10053000FA2010308400AD01AC004B210D300C1EB0
:100540009F2A99000A300C1EA32A990086300317AF
:100550008D0000308F000313B22083168C16C0303C
:1005600083128B042B08AB0AAC002C08AD001B30A7
:10057000AE002D08AF006430B000A4217708AD00B4
:1005800078083030031DCB2AAE1CD32AAE19D32AEB
:100590002E1A2030CE2AAE112E122E14F80778080B
:1005A0000C1ED02A99002D08AF000A30B000A421FB
:1005B0007708AD0078083030031DE42AAE19E92A27
:1005C0002E1CE92A2E1A2030F80778080C1EE62A7D
:1005D00099003030AD072D080C1EEC2A99007C30B4
:1005E0000C1EF02A99006430AC002C308400831378
:1005F00000080319082B0230F800F701F70BFE2A58
:10060000F80BFD2A9730F700F70B042B800BFB2A21
:08061000B22A8A150A16F32C28
:0C39E0000A128A11B9290A168A1508007B
:103A00008C1E002D1808A7001A08F800A71C0A2D04
:103A10001812181608008316B10803191F2D6530F7
:103A200083120C1E112D9900303083163207B3001B
:103A300083120C1E192D99008A0100288316831207
:103A400008008316B601B7013708013C031C552D49
:103A50003508FA003408840083137A1883170008A5
:103A6000403C0318422D360EB800F030B80534083B
:103A7000840083133518831700083807BF3E0A3EB9
:103A8000B6004F2D360EB800F030B805340884006B
:103A900083133518831700083807D03EB60037085F
:103AA000B70AB40A0319B50A242D3608F8008312A0
:103AB00008000B08F8008B138316031755308D0090
:103AC000AA308D008C14000000008C18652D0C119C
:103AD0007808831203138B040800831603178C17CE
:103AE00083120D08033903198A2DF9000D08FC39DA
:103AF0008D0083160C1483128D00000000008316C5
:103B00000C1583120313592503178D0A03198F0A05
:103B1000F90B7D2D831603133008F9000310F90CFF
:103B20000F30831203170D05031DA02D83160C16ED
:103B30000C15831203135925831603170C128312D5
:103B400000088C00840A00088E00840A83160C1575
:103B500083120313592503178D0A03198F0AF90BD2
:103B6000B22DB52D83160313902D0D0807390319B7
:103B7000C92D043CF900FF308C008E0083160C1513
:103B800083120313592503178D0A03198F0AF90BA2
:103B9000BB2D03130800E001DF010B138B138B1BFC
:103BA000CE2D40300C1ED22D990021300C1ED62D6A
:103BB00099008C1ADD2D6400D92D0D300C1EDE2DE0
:103BC00099000A300C1EE22D9900002578083A3C35
:103BD0000319EC2D6400E52D3A300C1EED2D9900F3
:103BE000AB012C302B0784008313EC010408EB009D
:103BF0006C10831B6C1400256B08840083136C18F5
:103C00008317780880002C302B078400831300086A
:103C1000E90069080C1E0A2E99002B08AB0A2C3EFD
:103C20008400831300080D3C03191A2E2B082D3C29
:103C30000318F12D2B082E3C0319202E0030212EC5
:103C40000130E9008316B1000130B20083120B2568
:103C50006400DA01E80103302B0268020318442EE5
:103C60002C306807E900EA010318EA0A6A0883169B
:103C7000B500831269088316B400831221257808E1
:103C8000DA070230E8072B2EDA08031D492E003030
:103C90004A2E0130E9008316B1000230B2008312CF
:103CA0000B258316B5012E30B40083122125780828
:103CB000E9008316B5013030B4008312212569086C
:103CC000DE007808DD008316B5013230B4008312BF
:103CD00021257808DC008316B5012C30B40083124E
:103CE00021257808DB005B08103C031C792E00308E
:103CF0007A2E0130E9008316B1000330B20083123E
:103D00000B255D08E1005E08E2000310E20CE10C07
:103D10005C0B902E23300C1E8B2E99008A010028FC
:103D2000DC08031D952E0030962E0130E900831625
:103D3000B1000430B20083120B25E801E601E50171
:103D40006208E4006108E3006808073C031CD42E05
:103D50000310680DA03E840083136608FA0065080E
:103D6000F9006408F8006308F7000130E30703185E
:103D7000E40A0319E50A0319E60A7A08EE0077084F
:103D800003178D000313780803178F0083168C1711
:103D90000C140000000083120C088000840A0E0836
:103DA00080000313E80AA42E0830E800E70105307C
:103DB0002B0268020318002F6708E70AA03EF800EC
:103DC000FA010318FA0A7808E9007A08EA002C30A8
:103DD0006807EB00EC010318EC0A6C088316B500C9
:103DE00083126B088316B4008312212569088400AE
:103DF00083136A188317780880000230E807D72EEB
:103E0000E108031D1F2FE208031D1F2F1C30E200D5
:103E1000F030E100620803178F00031361080317F5
:103E20008D00A03084008313103083160313B0007C
:103E300083126D2525300C1E1B2F9900492FE20897
:103E4000031D262F61080F3C0318452F62081C3CF8
:103E5000031C452F031D302F6108E03C031C452F38
:103E6000620803178F000313610803178D00A03049
:103E700084008313103083160313B00083126D2562
:103E800024300C1E412F9900492F2E300C1E462F36
:103E900099000D300C1E4A2F99000A300C1E4E2F2F
:103EA00099006400E52D0800AC01AB012B0F5B2FDE
:103EB0002C0F5B2F5F2FAB0A0319AC0A562F08009B
:103EC000840183131F308305713083168F000F0820
:103ED000031787110C3003139900A230980090301B
:103EE000831298008316031787110C30031399006F
:103EF000A2309800903083129800831603170908A7
:103F0000C039890003131F129F1200300317880065
:103F100083128701880189010313A701A801A90160
:103F20000B138B138B1B912F0930031785000F3058
:103F3000F700031381018130840083130008F039F6
:103F40000738800064000008F739F719F039770462
:103F50008000831603170908C039890003131F1254
:103F60009F12003003178800831203131F1083165B
:103F70000108C73908388100831290010030F80029
:103F80009200003083169200831203178701880184
:103F9000890183160313970171308F000F08831274
:103FA000AA012A0FD42FF82F8C1EE82F002578089D
:103FB000753C031DE72F2A300C1EDC2F99000025CD
:103FC0007808663C031DE62F6400CB25E82FF82F08
:103FD00075300C1EE92F990066300C1EED2F9900EC
:103FE0003F300C1EF12F990054276400AA0AD12FEC
:0C3FF00064001C308A00F0308200630086
:1000080000000000000000000000000000000000E8
:080018000000000000000000E0
:04400E00FD2CFF3F47
:00000001FF
